:020000021000EC
:10E000000C9446F00C9465F00C9465F00C9465F05B
:10E010000C9465F00C9465F00C9465F00C9465F02C
:10E020000C9465F00C9465F00C9465F00C9465F01C
:10E030000C9465F00C9465F00C9465F00C9465F00C
:10E040000C9465F00C9465F00C9465F00C9465F0FC
:10E050000C9465F00C9465F00C9465F00C9465F0EC
:10E060000C9465F00C9465F00C9465F00C9465F0DC
:10E070000C9465F00C9465F00C94ACF00C94F1F0F9
:10E080000C9465F00C9465F00C9465F011241FBE9F
:10E09000CFEFD0E1DEBFCDBF11E0A0E0B1E0E8ED11
:10E0A000F7EF01E00BBF02C007900D92A434B10757
:10E0B000D9F716E0A4E4B1E001C01D92AA3FB10770
:10E0C000E1F70E9467F00C94EAFB0C9400F00E94C8
:10E0D00057F187E089B988E18AB91124F89488ED6D
:10E0E00097EF9C01442737FD4095542FA0E0B1E005
:10E0F00008C04BBFF90187918D932F5F3F4F4F4F62
:10E100005F4F81E0A434B807A0F3E4E4F1E001C07C
:10E11000119286E0EA3FF807D8F381E380939C00F0
:10E120000E946FF882E380939C000E9427F383E3B0
:10E1300080939C000E94B3F1892B11F48BE201C003
:10E140008DE280939C0068EC70E080E090E00E949B
:10E150004AFA0C940000FFCF1F920F920FB60F9255
:10E160000BB60F9211242F933F938F939F93EF93AE
:10E17000FF9330919C00809149042091C30390E06B
:10E18000821B9109835E9F4FB4F3E091C303F0E0DB
:10E19000EF71F070E456F94F30838091C3038F5FC5
:10E1A0008093C30380919A00806280939A00E091EB
:10E1B0004401F0E0EF71F070E35BFE4F308380913B
:10E1C00044018F5F80934401FF91EF919F918F9164
:10E1D0003F912F910F900BBE0F900FBE0F901F908D
:10E1E00018951F920F920FB60F920BB60F92112433
:10E1F0008F939F93EF93FF939091C3038091490472
:10E20000981781F0E0914904F0E0EF71F070E45666
:10E21000F94F808180939C00809149048F5F8093A7
:10E22000490405C080919A008F7D80939A00FF91E8
:10E23000EF919F918F910F900BBE0F900FBE0F909B
:10E240001F901895382F809149042091C30390E0C6
:10E25000821B9109835E9F4FB4F3E091C303F0E00A
:10E26000EF71F070E456F94F30838091C3038F5FF4
:10E270008093C30380919A00806280939A0080E02B
:10E2800090E0089590914401809144049817D1F34F
:10E29000E0914404F0E0EF71F070E35BFE4F8081A9
:10E2A000909144049F5F9093440490E0089583E329
:10E2B0008093990088E980939A0082E291EF62E46A
:10E2C00071EF0E9476FA0895DF92EF92FF920F931A
:10E2D0001F93CF93DF93FC017B018A0181E04130E2
:10E2E000580710F000E011E081E0E03EF80798F5F3
:10E2F000FBBFDE2E80E09E2F63E00E9461FA80E08B
:10E3000090E061E10E9461FAC0E0D0E009C0F7014D
:10E31000EC0FFD1F60817181CE010E9463FA22968D
:10E32000C017D107A0F306C0CE016FEF7FEF0E94A8
:10E3300063FA2296CF3FD105B9F3B0F380E09D2D6B
:10E3400065E00E9461FA80E090E061E10E9461FA7C
:10E350008EE280939C00DF91CF911F910F91FF90EF
:10E36000EF90DF9008956F927F928F929F92AF927D
:10E37000BF92DF92EF92FF920F931F93CF93DF93A1
:10E3800081E090E0082E892F902D90937504809362
:10E390007404A6E7B4E002E010E0E4ECF3E081915D
:10E3A0008D930F5F1F4F8823D1F7FD018FE6819377
:10E3B00083E611968C93DF01119694E79183FD011A
:10E3C000319685E611968C939183128246E0842ED5
:10E3D000912C800E911E35E4A32EB12CEE24FF2447
:10E3E00024E0622E712CDD246091490170914A0174
:10E3F00080914B0190914C01A50120E034E0840113
:10E400000E94B7F497FD14C080E094E068E873E1DF
:10E410000E94D8F4EC018430910554F0809197016A
:10E4200090919801082E892F902D039731F064C0A8
:10E43000D39483E0D816C1F65FC0E114F10491F4DF
:10E44000A0908F01B09090010A2CAB2CB02CC3018E
:10E45000082E892F902D909375048093740494E076
:10E46000892E912C0091990110919A01002E012F73
:10E47000102DC70101960817190731F0E114F104B6
:10E4800009F43AC0870122C0C430D105B9F0EE0CBE
:10E49000FF1CAE0144505040C7016BE971E00E947F
:10E4A00064F181E0C530D8074CF0AE0144505140D2
:10E4B000C70101966BE972E00E9464F1C801082E61
:10E4C000892F902D9093770480937604C450D24086
:10E4D00014F0780188CF6091490170914A018091D0
:10E4E0004B0190914C01A50120E034E084010E9491
:10E4F000B7F420E030E002C02FEF3FEFC901DF9119
:10E50000CF911F910F91FF90EF90DF90BF90AF9050
:10E510009F908F907F906F900895DF93CF9300D05E
:10E5200000D0CDB7DEB7FC0119821A821B821C8293
:10E53000DE01119640E0808180538A3098F520E01A
:10E5400030E0C90163E0880F991F6A95E1F7220F57
:10E55000331F820F931F2191332727FD30952053BE
:10E560003040280F391F808180333CF08A332CF4EF
:10E570002F3F310531F328F315C02F3F310509F046
:10E5800088F44F5F2C9380818E3239F0443051F4FF
:10E5900029813A814B815C8109C0443019F0119680
:10E5A0003196C9CF2FEF3FEF4FEF5FEFB901CA01AF
:10E5B0000F900F900F900F90CF91DF910895CF9310
:10E5C000DF93982FE7E8F2E08081882301F18F3F05
:10E5D00001F1EF0121968917B1F49881491708F4E8
:10E5E000942FDF0120E030E009C0FB01E20FF31FB0
:10E5F00011968C91119780832F5F3F4F11962917A9
:10E60000A0F3888107C08181FE01E80FF11D3196DA
:10E61000DBCF80E0DF91CF910895CF93DF93FC01B2
:10E62000EA01322FDC016D9321831196922F03C0F2
:10E6300089918183915031969923D1F7FD01E30FA0
:10E64000F11D8FEF8083CF01DF91CF91089586E098
:10E6500091E00E948DF26093450170934601809392
:10E6600047019093480184E191E00E948DF260930C
:10E67000490170934A0180934B0190934C0182E2CF
:10E6800091E00E948DF26093BF037093C00380936A
:10E69000C1039093C20384EC93E060E371E00E94B5
:10E6A0006FFA80E090E00895AF92BF92CF92DF9230
:10E6B000EF92FF920F931F93DF93CF930F92CDB7FB
:10E6C000DEB76C01E62EFF245E010894A11CB11C8C
:10E6D0006FEF7FEF8FEF9FEF43E450E024E430E0F3
:10E6E00086010E94B7F497FD38C084E490E068E8A2
:10E6F00073E10E94D8F48C0197FD2FC00097F9F0C8
:10E7000020919B0130919C0140919D0150919E016F
:10E710008091780490917904A0917A04B0917B045F
:10E72000281739074A075B0751F485E3B50141E033
:10E730000E94DFF2813019F489818E1581F068EE34
:10E7400073E080E090E00E944AFAF39483E0F816C8
:10E7500009F0BECF00E010E002C00FEF1FEFC801CC
:10E760000F90CF91DF911F910F91FF90EF90DF906D
:10E77000CF90BF90AF9008950F931F93DF93CF93E7
:10E780000F92CDB7DEB721E02093740481E092E0D0
:10E79000A3E0B4E08093780490937904A0937A0482
:10E7A000B0937B0480E890E090937F0480937E0494
:10E7B0002093750486E08093760490E00AC0E92FE8
:10E7C000F0E0DF01A050BF4F8C91E057FB4F8083FA
:10E7D0009F5F9630A0F383E692E8A3E5B3E68093CB
:10E7E000600590936105A0936205B093630581E095
:10E7F000898384E695E065E38E010F5F1F4FA801D2
:10E8000021E00E940DF384EF90E062E00E9454F357
:10E81000181619060CF0A2C086E365E474E044E023
:10E820000E94DFF283E0898384E695E065E3A80136
:10E8300021E00E940DF362E347EA51E024E00E94E8
:10E840000DF366E345E454E024E00E940DF380E01C
:10E8500091E065E00E9454F3181619060CF07EC092
:10E860008091A7019091A801A091A901B091AA015E
:10E870008093450190934601A0934701B0934801CE
:10E8800086E091E00E948DF260934501709346010D
:10E89000809347019093480184E191E00E948DF2BA
:10E8A0006093490170934A0180934B0190934C010E
:10E8B00082E291E00E948DF26093BF037093C003E7
:10E8C0008093C1039093C2038091AB019091AC01FE
:10E8D000A091AD01B091AE018093490190934A019E
:10E8E000A0934B01B0934C010097A105B10581F4B1
:10E8F0008091870190918801A0918901B0918A014E
:10E900008093490190934A01A0934B01B0934C012D
:10E91000A3E0B2E0198280E007C0E82FF0E0EC53FA
:10E92000FC4F908311968F5F9C91992311F08F3744
:10E93000A0F38983E981F0E0EC53FC4F108281E081
:10E940006FEB73E044E00E94DFF286E365E474E07D
:10E9500044E00E94DFF220E030E002C02FEF3FEF02
:10E96000C9010F90CF91DF911F910F9108950F93DF
:10E970001F93022E232F302D30936D0420936C04AF
:10E98000042E452F502D50936F0440936E04085F62
:10E990001F4F9801022E232F302D309371042093A6
:10E9A000700441E198010E94FFF41F910F910895B6
:10E9B0000F931F93CF93DF938C01EB0181E1BE0195
:10E9C0000E9492F59C01181619069CF48091910101
:10E9D00090919201082E892F902D0817190771F731
:10E9E0002091930130919401022E232F302D285035
:10E9F0003040C901DF91CF911F910F910895BF92CF
:10EA0000CF92DF92EF92FF920F931F93DF93CF93FA
:10EA100000D000D000D0CDB7DEB77B018C01B42E82
:10EA20006901AE014F5F5F4F0E94C5F6892B19F057
:10EA30002FEF3FEF66C085E48093580484E190E0B7
:10EA4000C80ED91EC601082E892F902D90935B0405
:10EA500080935A0480E480936004B0926104E09251
:10EA60006804F092690400936A0410936B04809127
:10EA7000450190914601A0914701B09148018093D2
:10EA8000640490936504A0936604B0936704809136
:10EA90005C0490915D04019690935D0480935C0406
:10EAA0001092630410926204E8E5F4E020E030E0A4
:10EAB00040E050E081919191A0E0B0E0280F391F33
:10EAC0004A1F5B1F94E0EC36F907A1F705C0620FFF
:10EAD000731F9B0140E050E0CA01AA27BB27BC017D
:10EAE000892BA9F7C9018095909590936304809331
:10EAF0006204CE01019668E070E0A6010E94DAF798
:10EB00009C01C90126960FB6F894DEBF0FBECDBF9B
:10EB1000CF91DF911F910F91FF90EF90DF90CF90F9
:10EB2000BF9008951F93CF93DF93182FEB0188E0D8
:10EB300090E0BE010E944AF9BC01181619060CF0BB
:10EB400059C020917B01822F82958F70843079F794
:10EB50008091810190918201082E892F902D9F73C1
:10EB6000892B29F780918401811709F760917D0134
:10EB700070917E01062E672F702D822F8F7090E08E
:10EB8000880F991F880F991F681B790B20918B01A3
:10EB900030918C0140918D0150918E012F3F8FEF6C
:10EBA00038078FEF48078FEF580721F18091450113
:10EBB00090914601A0914701B09148010097A105AD
:10EBC000B10509F4B4CF281739074A075B0791F05C
:10EBD0008091BF039091C003A091C103B091C20383
:10EBE000282B392B4A2B5B2B2F5F3F4F4F4F5F4F0B
:10EBF00009F09DCFCB01DF91CF911F910895EF9246
:10EC0000FF920F931F93209145013091460140914F
:10EC10004701509148018091E2069091E306A0914E
:10EC2000E406B091E50682179307A407B50799F5A6
:10EC30008091D0069091D106082E892F902D0297B1
:10EC400009F09EC08091D8069091D906A091DA066D
:10EC5000B091DB068093E6069093E706A093E80662
:10EC6000B093E9068091D2068093EA068091D3069C
:10EC70008093EB068091D4068093EC068091D506B4
:10EC80008093ED068091D6068093EE068091D7069C
:10EC90008093EF0675C0E090D806F090D9060091F9
:10ECA000DA061091DB06E216F3060407150709F0F1
:10ECB00067C08091D0069091D106082E892F902DA3
:10ECC0008130910509F05CC0082E892F902D90931A
:10ECD000CB068093CA0688E090E09093CD0680939F
:10ECE000CC0686E08093CE0684E08093CF0682E057
:10ECF00090E0082E892F902D9093D1068093D00616
:10ED00008091D2068093DC068091D3068093DD0645
:10ED10008091D4068093DE068091D5068093DF062D
:10ED20008091D6068093E0068091D7068093E10615
:10ED3000E092E206F092E3060093E4061093E50603
:10ED4000809100018093D206809101018093D306C7
:10ED5000809102018093D406809103018093D506AF
:10ED6000809104018093D606809105018093D70697
:10ED700080E090E068E076E04CE150E00E94DAF755
:10ED80001F910F91FF90EF900895DF92EF92FF9205
:10ED90000F931F93CF93DF937B018C01EA018FEFD9
:10EDA000E8168FEFF8068FEF08078FEF180761F46A
:10EDB00080E090E02FEFFE01E80FF91F208301961D
:10EDC00086309105C1F7E4C08091E6069091E70690
:10EDD000A091E806B091E9068E159F05A007B1073E
:10EDE00009F4BDC021E030E0C901082E892F902D23
:10EDF0009093CB068093CA0688E090E09093CD066E
:10EE00008093CC0686E08093CE0684E08093CF0684
:10EE1000022E232F302D3093D1062093D0068091DF
:10EE200000018093D206809101018093D3068091E6
:10EE300002018093D406809103018093D5068091CE
:10EE400004018093D606809105018093D7068091B6
:10EE5000450190914601A0914701B09148018093EE
:10EE6000D8069093D906A093DA06B093DB068FEF0D
:10EE70008093DC068093DD068093DE068093DF06B8
:10EE80008093E0068093E106E092E206F092E306CA
:10EE90000093E4061093E506DD2480E090E068E04E
:10EEA00076E04CE150E00E94DAF797FD58C088E028
:10EEB00096E068EE73E00E944AF9181619060CF005
:10EEC00047C0209193013091940140919501509158
:10EED00096018091450190914601A0914701B09122
:10EEE0004801281739074A075B07A1F5809181017E
:10EEF00090918201082E892F902D029759F58091CB
:10EF0000890190918A01A0918B01B0918C0180932D
:10EF1000E6069093E706A093E806B093E906809191
:10EF200083018093EA06809184018093EB068091AF
:10EF300085018093EC06809186018093ED06809197
:10EF400087018093EE06809188018093EF0607C0C9
:10EF5000892B29F4D3948AE0D81609F09ECF8091AA
:10EF6000E6069091E706A091E806B091E9068E15B5
:10EF70009F05A007B10719F02FEF3FEF0BC0AAEED6
:10EF8000B6E0FE018D91819386E0A03FB807D1F7EE
:10EF900020E030E0C901DF91CF911F910F91FF90E8
:10EFA000EF90DF900895E199FECF9FBB8EBBE09A72
:10EFB0008DB30895EF92FF920F931F93CF93DF933A
:10EFC0007C0186E06830780719F00AE414E002C09A
:10EFD0000CEB16E0E801809100018E838091010125
:10EFE0008F838091020188878091030189878091B6
:10EFF00004018A87809105018B87E114F10481F077
:10F0000020E030E0FE01E20FF31FD701A20FB31F93
:10F010008C9180832F5F3F4F2630310599F707C0D1
:10F020008FEF888389838A838B838C838D837D870D
:10F030006C87425F5F4F4C33510510F0BA0102C03C
:10F040006CE370E082E2809300FFE62F60930AFF9A
:10F05000972F70930BFF109208FF80E4809309FFB5
:10F0600082E1809300FF20E030E007C0D8018D915D
:10F070008D01809310FF2F5F3F4F24173507B0F3AA
:10F0800004C0109210FF4F5F5F4F46175707C8F339
:10F0900082E2809300FF20E030E0809107FF86FD50
:10F0A00005C02F5F3F4F25313105B9F780E48093CC
:10F0B00007FFE09305FF909306FF809304FF86E22D
:10F0C000809300FF809100FF82FDFCCF80E090E004
:10F0D000DF91CF911F910F91FF90EF900895FF92D4
:10F0E0000F931F93E199FECF8DE490E09FBB8EBB01
:10F0F000E09A8DB380930301E199FECF8EE490E016
:10F100009FBB8EBBE09A8DB380930401E199FECF43
:10F110008FE490E09FBB8EBBE09A8DB38093050196
:10F1200010EC15BF00911FFF65E070E080E090E0FB
:10F130000E944AFA00931FFF68EE73E080E090E0BF
:10F140000E944AFA15BB14BB64E170E080E090E0D5
:10F150000E944AFA81EE809300FF80E4809301FFD1
:10F1600085B78F7785BF9D9903C08FEF9FEF0BC049
:10F170008FEF9FEF02C0009751F001979D99FBCF51
:10F18000F2CF009721F001979D9BFBCFECCF85B785
:10F19000806885BF15BA14BAF09000FF81E2F816B6
:10F1A000D9F710920FFF0FEF009307FF81EE8093C6
:10F1B00000FF80EC809301FF109206FF10E2109395
:10F1C00005FF109201FF68EC70E080E090E00E9483
:10F1D0004AFAF09200FF88E480930EFF10920AFF33
:10F1E00010920BFF10930CFF82E080930DFF80E4E0
:10F1F000809304FF8FE5809303FF9CE4909301FFCD
:10F2000080E6809302FF009307FF81E6809300FF72
:10F2100080910001809301FF80910101809302FFA2
:10F2200080910201809303FF80910301809304FF8A
:10F2300080910401809305FF80910501809306FF72
:10F24000109208FF109209FF10920AFF10920BFF14
:10F2500010920CFF10920DFF10920EFF10920FFFF4
:10F26000909307FFF09200FF84E080930CFF0093DF
:10F2700007FF10920FFF82E2809300FF10920DFFB4
:10F2800068EE73E080E090E00E944AFA1F910F91CF
:10F29000FF9008953F924F925F926F927F928F926C
:10F2A0009F92AF92BF92CF92DF92EF92FF920F9315
:10F2B0001F93DF93CF9300D000D0CDB7DEB76C01A2
:10F2C0007B0120E030E072E6372E02E264E0662E39
:10F2D0005AE0552E4E010894811C911C45E0A42E45
:10F2E000B12CAC0EBD1E90E4792E8FE5482EB1C036
:10F2F0009F5F409107FF42FDB4C040FD08C09923C5
:10F3000019F40894E108F108E114F10489F740FDCB
:10F3100003C0409307FFA7C0309200FF809107FF12
:10F32000009300FF109103FF1F5F103608F01CE4EC
:10F33000181719F4409307FF87C060920AFF1092D4
:10F340000BFF109208FF109309FF509200FF60E13D
:10F3500070E080E090E00E944AFAF401809110FF92
:10F360008193EA15FB05D1F7009300FF20E030E020
:10F37000809107FF86FD05C02F5F3F4F2531310586
:10F38000B9F7709207FF2B813C81C90180549040EE
:10F39000835B954018F00E946FF856C089818E708B
:10F3A00019F0B0E0A0E03BC0A90144505040B42F98
:10F3B000A52F40930AFF50930BFF609208FF109314
:10F3C00009FF509200FFBA0182E04335580710F060
:10F3D00062E572E0EDE6F1E020E030E005C080910A
:10F3E00010FF81932F5F3F4F26173707C0F39B0114
:10F3F00004C0809110FF2F5F3F4F24173507C8F3DB
:10F40000009300FF20E030E0809107FF86FD05C0FB
:10F410002F5F3F4F25313105B9F7709207FF8A8181
:10F4200081508A838C3408F44A828A81809303FF56
:10F430008091790190917A018C159D0539F0885061
:10F44000964011F40E94FFF5B0E0A0E08B2F9A2FB8
:10F450009C01E114F10439F02115310521F491E00A
:10F4600048CF2FEF3FEFC9010F900F900F900F90F3
:10F47000CF91DF911F910F91FF90EF90DF90CF9090
:10F48000BF90AF909F908F907F906F905F904F90C4
:10F490003F9008952BE0660F771F881F991F2A95CC
:10F4A000D1F720E030E040E050E005C000002F5FE1
:10F4B0003F4F4F4F5F4F2617370748075907B4F3A1
:10F4C0000895FC0103C0FC010B0161E0609368003A
:10F4D000E8956091680060FDFCCF11240895FB0160
:10F4E000DC0101900D920020E1F708950F931F9326
:10F4F000CF93DF938C01EB01009731F46115710517
:10F5000019F420E030E038C081E090E06EE070E077
:10F510000E94C2FAFC019C01009771F180E883838C
:10F52000209771F0D387C28781E883838091F006AA
:10F530009091F106892B21F4F093F106E093F00607
:10F5400001151105C9F011870087838182608383CB
:10F550008091F2069091F306892B71F4F093F306F3
:10F56000E093F2068091F4069091F506892B21F440
:10F57000F093F506E093F406C901DF91CF911F9156
:10F580000F9108950F931F93CF93DF93689F80018E
:10F59000699F100D789F100D1124C8010E94DEFA9A
:10F5A000EC01009729F060E070E0A8010E94E3FB05
:10F5B000CE01DF91CF911F910F910895CF93DF93EB
:10F5C000BC018230910510F462E070E0A091F80671
:10F5D000B091F906ED01E0E0F0E040E050E021C03C
:10F5E000888199818617970769F48A819B81309772
:10F5F00019F09383828304C09093F9068093F806F0
:10F60000FE0134C06817790738F44115510519F027
:10F610008417950708F4AC01FE018A819B819C0147
:10F62000E9012097E9F641155105A9F1CA01861BA8
:10F63000970B049708F4BA01E0E0F0E02AC08D913E
:10F640009C91119784179507F9F46417750781F455
:10F6500012968D919C911397309719F09383828322
:10F6600004C09093F9068093F806FD0132964FC0CE
:10F67000CA01861B970BFD01E80FF91F6193719377
:10F6800002978D939C9343C0FD01828193819C01DD
:10F69000D9011097A1F68091F6069091F706892B73
:10F6A00041F480913F01909140019093F70680933F
:10F6B000F60640914101509142014115510541F436
:10F6C0004DB75EB780913D0190913E01481B590BAB
:10F6D0002091F6063091F70624173507B0F4CA01D9
:10F6E000821B930B8617970780F0AB014E5F5F4F2D
:10F6F0008417950750F0420F531F5093F70640931D
:10F70000F606F9016193719302C0E0E0F0E0CF01E9
:10F71000DF91CF910895CF93DF93009709F450C004
:10F72000EC0122971B821A82A091F806B091F9068B
:10F73000109709F140E050E0AC17BD0708F1BB831A
:10F74000AA83FE0121913191E20FF31FAE17BF078B
:10F7500079F48D919C911197280F391F2E5F3F4F9F
:10F760003983288312968D919C9113979B838A836A
:10F770004115510571F4D093F906C093F80620C0E5
:10F7800012968D919C911397AD01009711F0DC01B9
:10F79000D3CFFA01D383C28321913191E20FF31FBA
:10F7A000CE17DF0769F488819981280F391F2E5FF2
:10F7B0003F4FFA01318320838A819B819383828327
:10F7C000DF91CF910895DC0101C06D93415050400D
:08F7D000E0F70895F894FFCF63
:10F7D8000006980101013139322E3136382E302E8B
:10F7E800313131003139322E3136382E302E313028
:10F7F80033003235352E3235352E3235352E300040
:10F808006669726D776172652E62696E002000FA12
:04F8180006000000E6
:040000031000E00009
:00000001FF
